:1000000011C0CFC9CEC9189518951895189518958F
:100010001895189518951895189518951895189578
:10002000189518958FE181BD87E181BD8FE58DBF62
:10003000C0E4E8E34E2E82E08EBFD2E0F2E05F2E15
:10004000EEEFF1E0A0E6B0E088278D933197E9F775
:1000500066248FEF8ABB8FEF84BB83EF81BB86E082
:1000600086B980E08093790080E080937A0081E017
:10007000809383008FEF80938100709178007F7D63
:1000800070937800709178007F777093780070910A
:1000900078007F7E7093780070917800777F7093FE
:1000A000780089B7806889BF81E38FBD89E08EBD04
:1000B00089E08093770052D98FEF809377004ED9F3
:1000C0006ED98BE08093770049D987E080937700E1
:1000D00045D965D98CE08093770040D981E0809341
:1000E00077003CD95CD98AE08093770037D98FE0DC
:1000F0008093770033D953D9C7D3E5D37091780073
:100100007068709378008BB780648BBF8BB7806802
:100110008BBF789485B78C7F836085BF85B7837FDD
:10012000886085BF929A939A389A85E090E0DDDBEB
:1001300038D480E080937900709178007860709373
:10014000780059D836D631DBA9DBA4E7B0E00C93B0
:100150004091740000917500041709F46EC000917D
:100160007400003109F469C000917400003009F096
:1001700004C081E08093760053C0013009F004C0D0
:1001800082E0809376004CC0023009F004C083E026
:100190008093760045C0043009F004C084E0809369
:1001A00076003EC0053009F004C085E080937600FB
:1001B00037C0063009F004C086E08093760030C076
:1001C000083009F004C087E08093760029C0093028
:1001D00009F004C088E08093760022C00A3009F05C
:1001E00004C089E0809376001BC00D3009F004C084
:1001F00080E08093760014C00C3009F004C08EE0DB
:10020000809376000DC00E3009F004C08FE080931B
:10021000760006C00F3009F003C08DE080937600B1
:10022000009176000D3009F407C07091780070617C
:100230007093780007D001C019D280917400809328
:10024000750082CF00917900003009F021C0009143
:1002500076000F3009F00AC081E08093790080E0D9
:1002600080937A00F8946ED2AFD20FC000917600DE
:100270000E3009F00AC081E08093790081E080931C
:100280007A00F8945FD2A0D2B8D2B5D70895A0C1B1
:10029000013009F064C000917A00003009F033C0E9
:1002A00000917600013009F008C082E08093790067
:1002B000809176008093660025C000917600023020
:1002C00081E008F480E08F9300917600093081E0AE
:1002D00010F009F080E09F918923882309F408C079
:1002E000809176008093650083E0809379000AC056
:1002F000009176000F3009F005C045D280E0809370
:100300007900789429C000917A00013009F024C066
:1003100000917600093010F009F008C082E0809367
:100320007900809176008093610016C0009176007C
:100330000E3009F008C082E08093790082E080935B
:100340007A006AD209C0009176000F3009F004C02B
:100350002BD580E0809379004ED7089539C10230C3
:1003600009F079C000917A00003009F03AC000919C
:100370007600043010F009F008C080917600809378
:10038000650083E0809379002BC0009176000530F2
:1003900081E008F480E08F9300917600093081E0DD
:1003A00010F009F080E09F918923882309F412C09E
:1003B00080916600809365008FE080936600809155
:1003C00076008093640084E08093790084E08093D9
:1003D000790006C0009176000F3009F001C0F9D015
:1003E00037C000917A00013009F009C08091760091
:1003F00080936000D6D280E08093790029C000917C
:100400007A00023009F024C000917600093010F023
:1004100009F008C083E08093790080917600809392
:10042000610016C0009176000E3009F008C083E02C
:100430008093790083E080937A00FDD109C0009118
:1004400076000F3009F004C0AFD480E080937900CB
:10045000D2D60895BDC0033009F053C000917A0090
:10046000003009F014C0009176000A3008F008C08E
:10047000809176008093640084E08093790006C0C8
:10048000009176000F3009F001C0A3D037C0009171
:100490007A00023009F009C08091760080936000F4
:1004A00047D380E08093790029C000917A0003301F
:1004B00009F024C000917600093010F009F008C05E
:1004C00084E080937900809176008093610016C06B
:1004D000009176000E3009F008C0BCD184E0809312
:1004E000790084E080937A0009C0009176000F3093
:1004F00009F004C059D480E0809379007CD6089537
:1005000067C0043009F03DC000917A00003009F066
:1005100014C0009176000A3008F008C0809176007F
:100520008093630085E08093790006C00091760097
:100530000F3009F001C04DD021C000917A00033086
:1005400009F009C080917600809360008FD380E02D
:100550008093790013C000917A00043009F00EC036
:10056000009176000E3009F005C0DED380E0809364
:10057000790004C019D480E0809379003CD60895B6
:1005800027C0053009F01BC000917A00003009F047
:1005900013C0009176000A3008F008C08091760000
:1005A0008093620086E08093790006C00091760017
:1005B0000F3009F001C00DD01ED6089509C00630D5
:1005C00009F006C000917A00003009F001C001D0A6
:1005D000089500917900013010F009F001C03FC08A
:1005E00000917900023009F00DC080E08093650031
:1005F00080E08093640080E08093630080E08093DB
:10060000620021C0033009F00AC080E080936400DA
:1006100080E08093630080E08093620014C0043027
:1006200009F007C080E08093630080E0809362005F
:100630000AC0053009F004C080E08093620003C066
:10064000063009F000C080E08093610080E0809374
:100650006000D1D5B9D5ADD380E080937900009109
:100660007900003009F001C0789408950027A8E7C8
:10067000B0E08C9185FB0EF401E041E0041709F035
:1006800006C080D1709178007F7D70937800A3E8D8
:10069000B0E08C918F5F8C9300918300053009F05E
:1006A00003C081E0809383005ED14CD08DE38093C2
:1006B000670087E48093660080E08093650080E0B7
:1006C0008093640000918300013009F00AC080EF3C
:1006D0008093630080E08093620081E080936100FA
:1006E00026C0023009F00AC080EF8093630081E0E9
:1006F0008093620080E08093610019C0033009F0AC
:100700000AC081EF8093630080E08093620080E004
:10071000809361000CC0043009F009C085EF80931C
:10072000630080E08093620080E08093610080E05D
:100730008093600060D527D07091780070627093CC
:100740007800089580916000809368008091610036
:10075000809369008091620080936A0080916300B9
:1007600080936B008091640080936C0080916500A1
:1007700080936D008091660080936E008091670089
:1007800080936F000895809168008093600080914D
:1007900069008093610080916A008093620080917B
:1007A0006B008093630080916C0080936400809163
:1007B0006D008093650080916E008093660080914B
:1007C0006F008093670008958FE0809360008FE052
:1007D000809361008FE0809362008FE080936300DC
:1007E0008FE0809364008FE0809365008FE08093BA
:1007F00066008FE0809367000895B5D08EE4809303
:10080000670087E7809366008EE0809365008EE046
:10081000809364008CD00895A6D08BE58093670008
:1008200087E7809366008EE3809365008FE4809372
:1008300064007DD0089597D08EE4809367008EE0A9
:10084000809366008FE48093650087E7809364005F
:100850006ED0089579D08EE4809367008EE0809307
:1008600066008FE48093650087E78093640081E0F1
:100870008093630087E7809362008EE0809361003D
:100880008EE08093600008955FD08BE580936700D1
:1008900081E0809366008EE3809365008FE480930F
:1008A000640085E08093630080E0809362008DEEB9
:1008B0008093610089E7809360009DD488EE93E087
:1008C00014D860D0089540D08BE5809367008FE402
:1008D000809366008FE58093650081E080936400DB
:1008E00080E3809363008EE7809362008EE78093BD
:1008F00061008DE3809360007ED488EB9BE0F5D7A8
:1009000041D0089530D08DE3809367008DE18093CE
:10091000660085E1809365008FE4809364008FE03A
:10092000809363008FE08093620065D408958FE028
:10093000809363008FE0809362008FE0809361007A
:100940008FE080936000089589E08093770006D55A
:1009500080E08093770002D522D5709178007F7770
:1009600070937800089589E080937700F7D48FE042
:1009700080937700F3D413D5709178007F777093CC
:100980007800089589E080937700E8D48FEF809312
:100990007700E4D404D57091780070687093780083
:1009A00008950027A8E7B0E08C9183FB0EF401E0E6
:1009B00041E0041709F005C01ED484EF91E095D7FB
:1009C00006C080E08093610080E080936000A1E633
:1009D000B0E00D9111274AE050E023D7ABE7B0E03B
:1009E0000D931C93ABE7B0E00D911C91A0E6B0E035
:1009F0004D915527040F151FABE7B0E00D931C93E5
:100A0000ABE7B0E00D911C9144E050E00AD7ABE7B2
:100A1000B0E00D931C93ABE7B0E0ED91FC91ADE736
:100A2000B0E091E0ACD7ABE7B0E0F5D6ABE7B0E033
:100A3000ED91FC91AEE7B0E091E0A1D7ABE7B0E07B
:100A4000EAD6ABE7B0E0ED91FC91AFE7B0E091E022
:100A500096D7ABE7B0E0DFD6ABE7B0E0ED91FC9125
:100A6000A0E8B0E091E08BD7ABE7B0E0D4D600913E
:100A70007D004FE00423A8E6B0E00C9300917D00D8
:100A800040EF0423A9E6B0E00C9394E0A9E6B0E0BF
:100A90003BD700917E004FE00423AAE6B0E00C9320
:100AA00000917E0040EF0423ABE6B0E00C9394E0AD
:100AB000ABE6B0E029D700917F004FE00423ACE61D
:100AC000B0E00C9300917F0040EF0423ADE6B0E06E
:100AD0000C9394E0ADE6B0E017D7009180004FE0B2
:100AE0000423AEE6B0E00C930091800040EF0423B5
:100AF000AFE6B0E00C9394E0AFE6B0E005D7002796
:100B0000A8E7B0E08C9183FB0EF401E041E004170C
:100B100009F004C0F7DE84EF91E0E7D633DF44D17B
:100B2000709178007061709378004ED342D108952F
:100B300062D384EF91E0D9D6A1E6B0E00D91112700
:100B40004AE050E06ED6ABE7B0E00D931C93ABE704
:100B5000B0E00D911C91A0E6B0E04D915527040F37
:100B6000151FABE7B0E00D931C93ABE7B0E00D9120
:100B70001C9144E050E055D6ABE7B0E00D931C93D8
:100B80008091690080937D0094E0ADE7B0E0D3D61A
:100B900000917D0040916800042BADE7B0E00C931C
:100BA00080916B0080937E0094E0AEE7B0E0C3D606
:100BB00000917E0040916A00042BAEE7B0E00C93F8
:100BC00080916D0080937F0094E0AFE7B0E0B3D6F2
:100BD00000917F0040916C00042BAFE7B0E00C93D4
:100BE00080916F008093800094E0A0E8B0E0A3D6ED
:100BF0000091800040916E00042BA0E8B0E00C93BF
:100C0000ABE7B0E0ED91FC91ADE7B0E091E07BE7C0
:100C1000A5D6ABE7B0E0FFD5ABE7B0E0ED91FC9136
:100C2000AEE7B0E091E07BE799D6ABE7B0E0F3D573
:100C3000ABE7B0E0ED91FC91AFE7B0E091E07BE78E
:100C40008DD6ABE7B0E0E7D5ABE7B0E0ED91FC9136
:100C5000A0E8B0E091E07BE781D6ABE7B0E0DBD580
:100C600051DE84EF91E041D69FD00895C4D284EF45
:100C700091E03BD6A1E6B0E00D9111274AE050E0AB
:100C8000D0D5ABE7B0E00D931C93ABE7B0E00D918E
:100C90001C91A0E6B0E04D915527040F151FABE75E
:100CA000B0E00D931C93ABE7B0E00D911C9144E0D4
:100CB00050E0B7D5ABE7B0E00D931C93ABE7B0E0E5
:100CC000ED91FC91A1E8B0E091E07BE747D6ABE77E
:100CD000B0E0A1D5ABE7B0E0ED91FC91A1E8B0E0C8
:100CE00091E07BE73BD6ABE7B0E095D5ABE7B0E072
:100CF000ED91FC91A1E8B0E091E07BE72FD6ABE766
:100D0000B0E089D5ABE7B0E0ED91FC91A1E8B0E0AF
:100D100091E07BE723D6ABE7B0E07DD5F3DD84EF50
:100D200091E0E3D541D00895EDDD84E090E0ADE8B9
:100D3000B0E08D939C93ADE8B0E00D911C910F381D
:100D400051E0150710F009F02DC0ADE8B0E0ED91CD
:100D5000FC91A1E8B0E091E07BE700D600918D0026
:100D600048E214D6A1E6B0E00C93ADE8B0E00D91F6
:100D70001C91003051E0150710F009F001C005C0CA
:100D8000A1E6B0E08C918A5F8C9300918D0048E2DF
:100D9000FDD5A0E6B0E08C932ED2ADE8B0E03BD517
:100DA00009F0C9CF01D00895EDDDEDDC24D27894AF
:100DB000089500916200003009F004C089E080933A
:100DC00070003EC0013009F004C088E080937000DC
:100DD00037C0023009F004C087E08093700030C053
:100DE000033009F004C086E08093700029C004300D
:100DF00009F004C085E08093700022C0053009F03E
:100E000004C084E0809370001BC0063009F004C069
:100E100083E08093700014C0073009F004C082E0C2
:100E2000809370000DC0083009F004C081E0809309
:100E3000700006C0093009F003C080E080937000A4
:100E400000916300003009F004C080E980937100D4
:100E50003EC0013009F004C080E88093710037C0C3
:100E6000023009F004C080E78093710030C0033085
:100E700009F004C080E68093710029C0043009F0B5
:100E800004C080E58093710022C0053009F004C0E1
:100E900080E4809371001BC0063009F004C080E339
:100EA0008093710014C0073009F004C080E2809381
:100EB00071000DC0083009F004C080E1809371001A
:100EC00006C0093009F003C080E0809371000091F2
:100ED0006400003009F004C089E0809372003EC0D5
:100EE000013009F004C088E08093720037C00230FE
:100EF00009F004C087E08093720030C0033009F02D
:100F000004C086E08093720029C0043009F004C058
:100F100085E08093720022C0053009F004C084E0AF
:100F2000809372001BC0063009F004C083E08093F8
:100F3000720014C0073009F004C082E08093720090
:100F40000DC0083009F004C081E08093720006C033
:100F5000093009F003C080E08093720000916600C0
:100F60000F3009F041C000916500013009F004C064
:100F700080EA8093730037C0023009F004C080E932
:100F80008093730030C0033009F004C080E8809380
:100F9000730029C0043009F004C080E78093730017
:100FA00022C0053009F004C080E6809373001BC0A6
:100FB000063009F004C080E58093730014C0073048
:100FC00009F004C080E4809373000DC0083009F07C
:100FD00004C080E38093730006C0093009F003C0A9
:100FE00080E280937300399A00916600013009F025
:100FF0002CC000916500003009F004C080E18093AE
:1010000073001BC0013009F004C080E080937300BE
:1010100014C0023009F004C080E2809373000DC058
:10102000033009F004C080E18093730006C00430EF
:1010300009F003C080E080937300009165000230E6
:1010400008F002C0399A01C03998009172004091AD
:101050007300042B0BBB0091700040917100042BB6
:1010600005BB8091660080938400009184000F305E
:1010700009F003C080E08093840094E0A4E8B0E02D
:1010800043D40091840040916500042BA4E8B0E0B3
:101090000C93A4E8B0E08C91A5E8B0E08D9388278C
:1010A0008C9398E0A5E8B0E039D4A5E8B0E00D91C4
:1010B0001C91A4E6B0E04D915527042B152BA5E813
:1010C000B0E00D931C93A5E8B0E00D911C910330A6
:1010D00052E0150708F003C0979896989598A5E8F0
:1010E000B0E00D911C91033052E0150781E008F447
:1010F00080E08F93A5E8B0E00D911C91053053E09E
:10110000150781E008F080E09F918923882309F486
:1011100003C097989698959AA5E8B0E00D911C9118
:10112000053053E0150781E008F480E08F93A5E8CF
:10113000B0E00D911C91033055E0150781E008F0F7
:1011400080E09F918923882309F403C09798969A99
:101150009598A5E8B0E00D911C91033055E0150776
:1011600081E008F480E08F93A5E8B0E00D911C9138
:10117000003058E0150781E008F080E09F91892356
:10118000882309F403C09798969A959AA5E8B0E049
:101190000D911C91003058E0150781E008F480E0C3
:1011A0008F93A5E8B0E00D911C91003055E1150733
:1011B00081E008F080E09F918923882309F403C02F
:1011C000979A9698959808950027A8E7B0E08C9193
:1011D00084FB0EF401E041E0041709F00BC0979A7C
:1011E0009698959A81E090E080D3709178007F7E08
:1011F0007093780008950027A8E7B0E08C9185FBF4
:101200000EF401E041E0041709F013C089E0809377
:101210007700A4D08FEF80937700A0D0C0D07091DA
:101220007800706870937800709178007F7D70937B
:10123000780088E0809382004091820001E00417EA
:1012400010F009F08AC0809182008093770086D0E8
:1012500000918200013009F005C080916000809308
:10126000770037C0023009F005C08091610080939B
:1012700077002FC0033009F005C080916200809391
:10128000770027C0043009F005C080916300809387
:1012900077001FC0053009F005C08091640080937D
:1012A000770017C0063009F005C080916500809373
:1012B00077000FC0073009F005C080916600809369
:1012C000770007C0083009F004C080916700809360
:1012D000770000918200063081E009F080E08F9372
:1012E0000027A8E7B0E08C9187FB0EF401E041E015
:1012F000041781E009F080E09F918923882309F495
:1013000005C0A7E7B0E08C9180518C9300918200DA
:10131000033081E009F080E08F930027A8E7B0E078
:101320008C9187FB0EF401E041E0041781E009F0A5
:1013300080E09F918923882309F405C0A7E7B0E0E6
:101340008C9180518C930AD02AD0809182008A950A
:10135000809382008F3F09F06FCF08959198889A0B
:101360008C9A9498A7E7B0E0119698E08E91983007
:1013700018F4392F992702C038E09850881F9098A8
:1013800008F4909A00000000949A000000009498DD
:10139000000000003A9591F7992341F70895919A3A
:1013A00008950F921F922F923F924F925F927F92D9
:1013B0008F929F92AF92BF920F931F932F933F9361
:1013C0004F935F936F937F938F939F93AF93BF934D
:1013D000CF93DF93EF93FF938FB78F930027BB27B4
:1013E000A5E28C9180FB0EF401E04427BB27A0E32B
:1013F0008C9182FB0EF44395041709F406C070919A
:10140000780070647093780005C0709178007F7BDD
:10141000709378001FD0EFDE8F918FBFFF91EF9117
:10142000DF91CF91BF91AF919F918F917F916F91FC
:101430005F914F913F912F911F910F91BF90AF906E
:101440009F908F907F905F904F903F902F901F9034
:101450000F9018950027A8E7B0E08C9186FB0EF45A
:1014600001E041E0041709F0EDC000918300013074
:1014700009F006C0809160008A958093600029C0C1
:10148000023009F009C0809161008A958093610063
:1014900080E0809360001DC0033009F00CC0809193
:1014A00062008A958093620080E08093610080E012
:1014B000809360000EC0043009F00BC0A2E6B0E0DB
:1014C0008C9185508C9380E08093610080E08093C4
:1014D0006000009160000F3F09F008C089E0809330
:1014E0006000809161008A958093610000916100A5
:1014F0000F3F09F008C089E080936100809162008D
:101500008A958093620000918300043081E009F0A5
:1015100080E08F93009162000F3F81E010F009F0AE
:1015200080E09F9189238F9300916200003F80E0CB
:1015300010F009F081E09F918923882309F40EC0FF
:1015400085E080936200809163008A9580936300B8
:10155000709178007061709378002AC000918300C8
:10156000043081E009F480E08F93009162000F3F26
:1015700081E010F009F080E09F9189238F93009122
:101580006200003F80E010F009F081E09F91892324
:10159000882309F40DC089E0809362008091630084
:1015A0008A958093630070917800706170937800E1
:1015B000009163000F3F09F008C089E08093630049
:1015C000809164008A9580936400009164000F3FCD
:1015D00009F008C089E080936400809165008A95D5
:1015E0008093650000916500003081E009F080E0A3
:1015F0008F93009166000F3081E009F080E09F91A9
:101600008923882309F412C080E08093600080E081
:101610008093610080E08093620080E080936300AB
:1016200080E08093640081E0809365000091650014
:101630000F3F09F006C08FE08093660089E0809339
:101640006500AFC000918300013009F006C0A0E63C
:10165000B0E08C918F5F8C9329C0023009F009C0F3
:10166000A1E6B0E08C918F5F8C9380E08093600066
:101670001DC0033009F00CC0A2E6B0E08C918F5F72
:101680008C9380E08093610080E0809360000EC0C6
:10169000043009F00BC0A2E6B0E08C918B5F8C9314
:1016A00080E08093610080E08093600000916000A2
:1016B0000A3009F008C080E080936000A1E6B0E045
:1016C0008C918F5F8C93009161000A3009F008C003
:1016D00080E080936100A2E6B0E08C918F5F8C93F4
:1016E000009162000A3008F40DC080E0809362002F
:1016F000A3E6B0E08C918F5F8C937091780070615D
:1017000070937800009163000A3009F008C080E00F
:1017100080936300A4E6B0E08C918F5F8C9300917E
:1017200064000A3009F008C080E080936400A5E6F8
:10173000B0E08C918F5F8C93009165000A3009F0C6
:1017400006C080E08093650081E080936600009190
:101750006600013081E009F080E08F930091650020
:10176000053081E008F480E09F918923882309F403
:1017700018C08FE08093670081E08093660084E06A
:101780008093650089E08093640089E08093630022
:1017900089E08093620089E08093610089E0809312
:1017A000600012DD06DB01D00895A0E6B0E09C9158
:1017B00065D0A9E8B0E08D9388278C93A1E6B0E0CE
:1017C0009C915CD0082F11274AE050E02AD0ABE86A
:1017D000B0E00D931C93ABE8B0E00D911C91A9E82B
:1017E000B0E04D915C91040F151FA7E8B0E00D9398
:1017F0001C93A7E8B0E00D911C9142E050E011D09D
:10180000A7E8B0E00D931C93A7E8B0E08C9188BDE9
:101810000895F894FFCFED91FC913196FC93EE93EF
:10182000089504D01FD000FC0CD008950024E89443
:1018300057FF02C009D0689400F80BD010F80124BB
:10184000089502D009D00895509540954F5F5F4F9D
:101850000895E89417FF0895009510950F5F1F4FA6
:10186000689408950F92049F202C312C419F300CD6
:10187000509F030C022D102D0F900895892F8F700B
:10188000905110F0865FFCCF08953197F1F70895DD
:10189000689462F80895E89462F8089500E18FEF83
:1018A00088BB8FE087BB80EF88BB84E68A95F1F721
:1018B000B49B00E0B59B04E0B69B08E0B79B0CE04E
:1018C00080EF87BB8FE088BB84E68A95F1F7882795
:1018D000B09B80E0B19B81E0B29B82E0B39B83E050
:1018E000080F84E690E001D00895EF93FF93EE2770
:1018F000E82BE92B31F0E4ECF9E03197F1F70197AF
:10190000D1F7FF91EF910895903039F08C91880FC5
:1019100008F481609A95D9F78C930895903051F02E
:1019200000240D911C91000F111F001D9A95D9F7ED
:101930001C930E930895903039F08C91869508F49D
:1019400080689A95D9F78C930895E199FECFEEBB04
:10195000FFBB3196089591E001C092E07B3751F4CE
:101960007FB7F894F2DF8D918DBBE29AE19A9A9558
:10197000C9F77FBF7727089591E001C092E0E5DFC6
:10198000E09A8DB38D939A95D1F70895FF93881BB4
:10199000F9E0001FFA9511F4FF910895881F841B48
:0C19A00018F4840F8894F5CF0894F3CF5E
:00000001FF
